:100000000C9434000C9449000C9449000C94490061
:100010000C9449000C9449000C9449000C9449003C
:100020000C9449000C9449000C9449000C9449002C
:100030000C9449000C9449000C9449000C9449001C
:100040000C9449000C9449000C9449000C9449000C
:100050000C9449000C9449000C9449000C944900FC
:100060000C9449000C94490011241FBECFEFD4E03A
:10007000DEBFCDBF11E0A0E0B1E0E0E2F3E002C0FE
:1000800005900D92AE30B107D9F70E9474010C941F
:100090008E010C9400008AB1806E8AB980910001B3
:1000A00081FF03C08BB18F7102C08BB1806E8BB9A1
:1000B00008958093000108950C944B00982F80912F
:1000C00000014BB121E030E0B90102C0660F771F9B
:1000D0009A95E2F781FF04C0CB018095842302C08A
:1000E000CB01842B8BB90895982F809100014BB1DF
:1000F00021E030E0B90102C0660F771F9A95E2F760
:1001000081FF03C0CB01842B03C0CB0180958423E6
:100110008BB90895CF93C82F0E9474008FE19EE49D
:100120000197F1F700C000008C2F0E945E009FEF46
:100130002AE683E0915020408040E1F700C00000B3
:10014000CF91089585E00E948A0086E00E948A008F
:1001500087E00C948A00459A85E38A95F1F70000C0
:100160004598089598B1907F98B998B182958F700D
:10017000982B98B90C94AB00CF93C82F449A0E9447
:10018000B2008C2F8295807F0E94B2008AE78A9508
:10019000F1F700C0CF910895CF93C82F44980E94E3
:1001A000B2008C2F8295807F0E94B20080E78A95F2
:1001B000F1F7CF91089581E00E94CC008FE99FE094
:1001C0000197F1F700C00000089587B18F6387B9E8
:1001D00088B1807C88B98FE295E70197F1F700C07C
:1001E000000080E30E94B2008FE097E20197F1F7F0
:1001F00000C000000E94AB008FEC97E00197F1F780
:1002000000C000000E94AB008FEC97E00197F1F76F
:1002100000C0000080E20E94B2008FE097E20197E8
:10022000F1F700C0000088E20E94CC008CE00E9440
:10023000CC0086E00E94CC000C94DB0082E00E949F
:10024000CC008FE99FE00197F1F700C0000008950E
:10025000623059F018F4613031F00895633039F0AC
:10026000643039F00895805805C0805403C0805729
:1002700001C080530C94CC00CF93DF93EC018991A3
:10028000882319F00E94BC00FACFDF91CF91089526
:10029000EF92FF920F931F93CF93DF9300D0CDB7D0
:1002A000DEB728E0829FC0011124806469837A83CD
:1002B0000E94CC006981E62E7A81F72E8701085FC3
:1002C0001F4FF70181917F010E94BC00E016F106EB
:1002D000C1F780E80F900F90DF91CF911F910F91A0
:1002E000FF90EF900C94CC0081E00E9459000E9496
:1002F0005C000E94A2000E94E50081E091E00E9463
:100300003C0185E00E948A002FEF89E698E12150A8
:1003100080409040E1F700C00000F3CFF894FFCF99
:0E03200001497420776F726B27732100000073
:00000001FF
